:020000040800F2
:100000003005002001010008250100082701000833
:10001000290100082B0100082D0100080000000044
:100020000000000000000000000000002F01000898
:10003000310100080000000033010008350100080C
:1000400037010008370100083701000837010008B0
:1000500037010008370100083701000837010008A0
:100060003701000837010008370100083701000890
:100070003701000837010008370100083701000880
:100080003701000837010008370100083701000870
:100090003701000837010008370100083701000860
:1000A0003701000837010008370100083701000850
:1000B0003701000837010008370100083701000840
:1000C0003701000837010008370100083701000830
:1000D0003701000837010008370100083701000820
:1000E000370100083701000837010008DFF80CD09D
:1000F00000F02CF800480047F90100083005002006
:100100000D488047DFF83400016841F4E0210160C8
:10011000BFF34F8FDFF82800DFF8281001600A488E
:1001200000477047FEE7FEE7FEE7FEE7FEE7FEE773
:10013000FEE7FEE7FEE7FEE72301000824ED00E00E
:100140000CED00E00003FA05ED000008064C074D39
:1001500006E0E06840F0010394E807009847103497
:10016000AC42F6D3FFF7C6FF480200086802000859
:1001700070B58D1810F8014B14F0030201D110F87E
:10018000012B231106D110F8013B03E010F8016B9D
:1001900001F8016B521EF9D1ABB110F8012B04F03C
:1001A0000C048A1A0C2C03D0A2EB84129B1C08E0CE
:1001B00010F8014BA2EB0422F8E712F8014B01F80A
:1001C000014B5B1EF9D5A942D4D3002070BD40F28B
:1001D000010CC2F2000C604702E008C8121F08C1FF
:1001E000002AFAD170477047002001E001C1121FB8
:1001F000002AFBD17047000010B5002419E020460A
:10020000FFF7E5FF0D490860084600680C490968DA
:10021000884203DD0948006809490860074800680A
:1002200008490968884203DA0448006805490860FB
:10023000641C402CE3DB002010BD000028000020DF
:100240002000002024000020680200080000002098
:100250002C010000700100081C0300082C01002084
:1002600004040000E80100083007054B33F91010C2
:100270000610132001FB01F102FB02107047000081
:10028000AC0000202C04100900000080FFFFFF7F5D
:100290000800821E00FF7F627F8A7D7D7A4276E3BE
:1002A000706E6AF262825A34511D47573CFC302806
:1002B00025F9188C0C000074F307E7D8DA04CFA9ED
:1002C000C3E3B8CCAE7EA50E9D92951D8FBE8983EB
:1002D0008576829E8000809E8076828385BE891D81
:1002E0008F92950E9D7EA5CCAEE3B8A9C304CFD85E
:1002F000DA07E774F300008C0CF9182825FC305756
:100300003C1D473451825AF2626E6AE37042767D38
:0C0310007A8A7D627F20015EA000000060
:04000005080000ED02
:00000001FF
